:100000000C9463000C9450080C947D080C948B00A5
:100010000C948B000C948B000C948B000C948B0034
:100020000C948B000C948B000C948B000C948B0024
:100030000C948B000C948B000C948B000C948B0014
:100040000C94AA080C948B000C94860B0C94B80B9F
:100050000C948B000C948B000C948B000C948B00F4
:100060000C948B000C948B0000000008000201002F
:100070000003040700000000000000000102040863
:100080001020408001020408102001020408102002
:10009000040404040404040402020202020203032E
:1000A00003030303000000002300260029000000D2
:1000B0000000250028002B0000000000240027007D
:1000C0002A00A300E80B11241FBECFEFD8E0DEBF4B
:1000D000CDBF11E0A0E0B1E0E2E3FBE102C005909A
:1000E0000D92A63CB107D9F723E0A6ECB1E001C020
:1000F0001D92AE30B207E1F710E0C6ECD0E004C0CC
:100100002297FE010E94930DC23CD107C9F70E94BD
:100110002C0C0C94970D0C9400001F93CF93DF933D
:10012000182FEB0161E00E94E809BE01882777FDE6
:100130008095982F0E94230960E0812FDF91CF9155
:100140001F910C94E80920E042E06AE086E092E02A
:100150000C940A0226E040E855E260E070E081E796
:1001600092E00E942A0B66E071E081E792E00E9433
:10017000790C4AE050E061E070E081E792E00E9493
:100180003B0D6CE071E081E792E00E94860C61E03B
:100190008EE00E94AF0960E08EE00E94E80920E056
:1001A00041E050E06BE586E092E00E94A30461E04C
:1001B00086E092E00E94C00763E171E086E092E091
:1001C0000C945E04EF920F93CF9381E792E00E942C
:1001D000470A181619060CF067C081E792E00E94E2
:1001E000600A8D30B1F464E271E081E792E00E9430
:1001F000790C4AE050E062E070E081E792E00E9412
:100200003B0D65E371E081E792E00E94790CC0E06C
:1002100011C02091040230910502F901EA53FE4F0A
:100220008083C90101969093050280930402CD97C3
:10023000D9F5D9CF8C2F90E020910402309105029E
:100240008217930754F4FC01EA53FE4F608181E763
:1002500092E00E947B0CCF5FEDCF61E471E081E71B
:1002600092E00E94860C8EE1E82E02E020910402CA
:1002700046EC51E062E070E086E092E00E943A02D3
:10028000882319F063E471E002C061E571E081E761
:1002900092E00E94860C10920502109204026AE01D
:1002A00070E08EE00E948D0086E092E00E94E206FF
:1002B000882309F451C061E671E081E792E00E9471
:1002C000790C60911E0270911F024AE050E081E7B4
:1002D00092E00E94680D65E371E081E792E00E9480
:1002E000790CC0E080912002C81758F4EC2FF0E0A0
:1002F000EE5DFD4F608181E792E00E947B0CCF5F55
:10030000F1CF65E771E081E792E00E94790C60919E
:100310001702709118024AE050E081E792E00E94D3
:10032000430D86E092E00E948F02882369F040E04E
:1003300067EB71E086E092E00E945A076EE771E099
:1003400081E792E00E94860C6AE070E08EE0CF9137
:100350000F91EF900C948D00CF910F91EF90089535
:10036000089581E0809316020895CF93DF93EC0106
:1003700061E08A810E94E80980916202882361F02D
:100380009FB7F8942091620280916002213019F4A5
:100390008DBB9FBF01C08FBF8A858CBD8B858DBDF6
:1003A000DF91CF910895FC018CB582878DB583874D
:1003B0003485258580916202882399F09FB7F8944F
:1003C00080916202813059F48DB3809360024DB305
:1003D00080916102809584238DBB9FBF02C0909362
:1003E00060023CBD2DBD8CB5837F8CBD8CB58F7DEF
:1003F0008CBD8CB58C7F8CBD8DB58E7F8DBD60E046
:1004000082810C94E8098EBD00000DB407FEFDCF7B
:100410008EB50895FC018BE891E09183808380E59F
:10042000848781E0858762834383809321021782DA
:100430008FE1808721870895CF93DF93EB01DC0163
:10044000ED91FC910480F581E02D0995882371F0F0
:1004500080911E0290911F028C179D0711F0CD2BE9
:1004600029F481E090911902911101C080E0DF919F
:10047000CF9108952F923F924F925F926F927F9209
:100480008F929F92AF92BF92CF92DF92EF92FF92A4
:100490000F931F93CF93DF93EC015B014A01722E00
:1004A000602E10E0CE2CD12CE12CF12CE881F981CA
:1004B0000190F081E02D01E0272DA401B501CE01CE
:1004C00009950E94F4081B012C010E94F40862198E
:1004D0007309840995096C157D058E059F0540F407
:1004E000B501CE010E941C02882379F381E004C08B
:1004F0001F5F6116D8F680E0DF91CF911F910F91B9
:10050000FF90EF90DF90CF90BF90AF909F908F9033
:100510007F906F905F904F903F902F9008958091C3
:100520001A02882339F081E020911C0230911D02CB
:10053000232B09F480E00895EF92FF921F93CF934D
:10054000DF931F92CDB7DEB77C01DC01ED91FC910A
:100550000688F789E02D698309956981862F8F7751
:100560000E94030280E00E940302182FD701ED9140
:10057000FC91008CF18DE02DC7010995812F0F9022
:10058000DF91CF911F91FF90EF9008950F931F93EC
:10059000CF93DF9300D0CDB7DEB78C01DC01ED91B6
:1005A000FC910688F789E02D4A8369830995698162
:1005B000862F80680E9403024A81842F0E940302D2
:1005C000D801ED91FC91008CF18DE02DC8010F90C8
:1005D0000F90DF91CF911F910F9109941F93CF93AB
:1005E000DF93EC01162F80912102681709F461C096
:1005F000623009F440C070F4662309F444C06130ED
:1006000009F057C061E0CE010E949C02482F437E52
:1006100044603FC06330C1F0643009F04AC061E01B
:10062000CE010E949C02482F437E4C6061E0CE01C7
:100630000E94C6028985882381F1E881F9810488B6
:10064000F589E02D61E014C061E0CE010E949C02BA
:10065000482F437E406161E0CE010E94C602898539
:100660008823D9F0E881F9810488F589E02D60E0DC
:10067000CE01099512C061E0CE010E949C02482F74
:10068000437E486006C061E0CE010E949C02482F74
:10069000437E61E0CE010E94C60280912102811159
:1006A00006C067E2CE010E949C0287FFF6CF10933E
:1006B0002102DF91CF911F910895CF93DF93EC0139
:1006C000603208F06FE168878985882311F06695AC
:1006D000688761E1CE010E949C02482F407E888598
:1006E000482B61E1CE01DF91CF910C94C6028F922D
:1006F0009F92AF92BF92CF92DF92EF92FF920F93B1
:100700001F93CF93DF931F92CDB7DEB74C016B01E0
:10071000142FB52EF22EA02EDC01ED91FC91028853
:10072000F389E02D61E0099567E2C4010E949C0213
:1007300087FFFACF40E065E2C4010E94C6020F2D98
:100740000E3308F00DE3E11004C0A11004C020E056
:1007500003C020E801C020E4BFEFCB16D10451F064
:1007600048F0B6016627737056E0769567955A95FE
:10077000E1F7262BF401658176816F3F710521F049
:1007800018F066277370272BD401ED91FC91068831
:10079000F789E02DC4012983099580E80E940302AE
:1007A00083E0800F0E9403028C2D0E940302F4015B
:1007B00085810E9403022981822F0E940302D12E8B
:1007C000E12EFB2C8E2D8D19801730F4D7018D91E1
:1007D0007D010E940302F6CFD401ED91FC91008CC3
:1007E000F18DE02DC4010995D401ED91FC910288B1
:1007F000F389E02D64E0C40109950E94F4086B01BF
:100800007C01F40183810E941E0A892BB1F0D4017E
:10081000ED91FC910288F389E02D61E0C4010F9015
:10082000DF91CF911F910F91FF90EF90DF90CF90CC
:10083000BF90AF909F908F9009940E94F4086C191C
:100840007D098E099F09683E734081059105F8F680
:10085000D8CFCF93DF93EC011092200210921F02A9
:1008600010921E0210921D0210921C0210921B0286
:1008700010921A0210921902109218021092170286
:1008800068E20E949C0282FF0AC06DE3CE010E94D2
:100890009C02482F44606DE3CE010E94C60240E4F2
:1008A00065E2CE010E94C602E881F9810288F389DF
:1008B000E02D63E0CE01DF91CF910994DF92EF92BA
:1008C000FF920F931F93CF93DF93EC018B01E8818D
:1008D000F9810288F389E02D61E009950115110580
:1008E000E1F0E881F9810688F789E02DCE010995CC
:1008F0008EEB0E9403027801D12CF70181917F01D8
:100900000E940302D394F0E1DF12F7CFE881F9816E
:10091000008CF18DE02DCE0109956DE3CE010E9492
:100920009C028E7F91E0012B09F490E0482F492B27
:100930006DE3CE01DF91CF911F910F91FF90EF906A
:10094000DF900C94C6028F929F92AF92BF92CF928B
:10095000DF92EF92FF920F931F93CF93DF93CDB768
:10096000DEB7AE970FB6F894DEBF0FBECDBF7C01E9
:100970006A01DC0113968C91823021F0833021F4DE
:1009800081E003C080E001C08FEFF70184838EE235
:100990008E010F5F1F4FD801E82F1D92EA95E9F7EE
:1009A00091E0998334E03A8342E04B8393E09D8366
:1009B0004E833F8340E4488735E039879A8796E045
:1009C0009B8793E39C8737E03D8798E09F8799E07A
:1009D000998B99E19B8B92E49C8B55E25D8B4E8BBE
:1009E00046E24F8B388F38E2398F30E13A8F39E267
:1009F0003B8F3CED3C8F8D8F88E88E8F8FE28F8F01
:100A00008DE288A380E389A337E33BA330E93CA3CD
:100A100038E33DA39EA39CE39FA39FE898A79DE393
:100A200099A792E19AA79FE69BA78CA78FEF8DA726
:100A30006F3131F06B3231F0663531F489ED05C03C
:100A40008EE403C08CE601C084EE8E876F3141F0E6
:100A50006B3221F0663521F480E003C080E401C0F0
:100A600080EC888B2AA361E0D70112968C910E94BA
:100A7000E80961E0F70182810E94AF090E94FA074C
:100A800080E5D7011C968C931C9781E01D968C9372
:100A90000E94F4084B015C014AEA6FE2C7010E9420
:100AA000C6026FE2C7010E949C028A3A59F00E9476
:100AB000F408681979098A099B096233710581056F
:100AC000910550F30E94F4084B015C0145E56FE28B
:100AD000C7010E94C6026FE2C7010E949C028535D1
:100AE00059F00E94F408681979098A099B09623350
:100AF00071058105910550F3B12CF801EB0DF11D45
:100B0000EB0DF11D60816F3F31F04181C7010E9403
:100B1000C602B394F2CF60E070E0C7010E945E04A9
:100B2000D701ED91FC9111970084F185E02D199684
:100B30006C91C7010995D701ED91FC910288F38969
:100B4000E02D61E0C70109950E94F4084B015C01AA
:100B500067E2C7010E949C0287FD0BC00E94F40857
:100B6000681979098A099B09623371058105910524
:100B700078F30E94F408681979098A099B0962339D
:100B800071058105910598F443E050E061EB71E057
:100B9000F70184810E943008F0921502E09214025D
:100BA000D7011696DC92CE92159781E001C080E0C5
:100BB000AE960FB6F894DEBF0FBECDBFDF91CF91DA
:100BC0001F910F91FF90EF90DF90CF90BF90AF906B
:100BD0009F908F900895CF93DF93EC0161110DC02A
:100BE00064E2CE010E949C0290E09195819591096A
:100BF00095958795DF91CF91089541E063E20E943A
:100C0000C60263E2CE010E949C0281FFFACFE8CFC8
:100C1000CF93DF93EC01809121028330A9F480917E
:100C20001B02811111C060E0CE010E94EB05863AE3
:100C30009F4F54F4E881F9810288F389E02D61E047
:100C4000CE01099581E001C080E0DF91CF91089548
:100C50001F93CF93DF93EC01809121028330D1F475
:100C600068E2CE010E949C0282FD20C013C0F0E029
:100C7000EE5DFD4F1082E881F981008CF18DE02D51
:100C8000CE010995E881F9810288F389E02D63E0BE
:100C9000CE01099560E0CE010E94EB059093180209
:100CA00080931702DF91CF911F910895E881F98118
:100CB0000288F389E02D61E0CE010995E881F98190
:100CC0000688F789E02DCE01099580E00E94030295
:100CD00080E00E940302833408F082E480931B02C8
:100CE00080E00E94030290E090931D0280931C021A
:100CF00080E00E94030290E090931F0280931E0206
:100D000080E00E940302282F2C7090E4299F90011C
:100D1000112440911C0250911D02242B352B30933D
:100D20001D0220931C02982F937040911E02509137
:100D30001F02592B50931F0240931E029F81911155
:100D400007C04D815E812417350711F0232B21F454
:100D500090911B02933098F410921B02E881F98164
:100D6000008CF18DE02DCE010995E881F981008894
:100D7000F189E02DCE01DF91CF911F91099493501D
:100D800090932002982F907890931902982F907446
:100D900090931A02E881F9810484F585E02D682F8B
:100DA000CE01099510E0E09120021E1708F05FCFF8
:100DB00080E00E940302E12FF0E0EE5DFD4F8083B2
:100DC0001F5FF1CFCF93DF93EC0180911602882350
:100DD00029F010921602CE010E942806809121026D
:100DE000833071F480911B02882389F0E881F981B6
:100DF0000288F389E02D61E0CE01099581E008C009
:100E0000E881F9810088F189E02DCE01099580E023
:100E1000DF91CF9108954F925F926F927F928F9260
:100E20009F92AF92BF92EF920F931F93CF93DF9356
:100E3000EC015B014A01122F6DE30E949C02482FD6
:100E400044606DE3CE010E94C6020E94F4082B01AB
:100E50003C01CE010E9408068823C9F0E881F9818F
:100E60000684F785E02DE12C212FA401B501CE01E8
:100E70000995DF91CF911F910F91EF90BF90AF90A7
:100E80009F908F907F906F905F904F9008950E94F9
:100E9000F4086419750986099709683E734081054D
:100EA0009105E0F6E881F9810480F581E02DCE011D
:100EB0000995CFCF4F925F926F927F928F929F92C0
:100EC000AF92BF92CF92DF92EF920F931F93CF9387
:100ED000DF93EC014B01142F10921A02C0901E02F6
:100EE000D0901F02A0901702B09018026DE30E94EC
:100EF0009C02482F44606DE3CE010E94C6020E940E
:100F0000F4082B013C01CE010E940806882329F138
:100F1000D0921F02C0921E02E881F9810684F785F3
:100F2000E02DEE24E39400E0212FA401B601CE01D0
:100F30000995B0921802A0921702DF91CF911F91EC
:100F40000F91EF90DF90CF90BF90AF909F908F90D8
:100F50007F906F905F904F9008950E94F4086419FD
:100F6000750986099709683E73408105910580F6E9
:100F7000E881F9810480F581E02DCE010995C3CF88
:100F8000CF93DF93EC016987662311F04FE001C036
:100F90004AE163E1CE010E94C6028985882341F0BF
:100FA00061E1CE010E949C02482F4F71406602C051
:100FB0004885406861E1CE01DF91CF910C94C60273
:100FC0001F93CF93DF93EC01162F662311F04DE5AD
:100FD00001C045E56AE5CE010E94C602112311F069
:100FE0004CE701C040E76CE5CE01DF91CF911F9146
:100FF0000C94C602CF93CFB7F8948091630281110D
:1010000027C0EAE9F0E08491E6E8F0E09491E82F67
:10101000F0E0EE0FFF1FE854FF4FA591B4918C91C3
:10102000892321F461E08AE00E94E80961E08AE016
:101030000E94AF098CB580618CBD8CB580648CBD7D
:1010400061E08DE00E94AF0961E08BE00E94AF0992
:10105000809163028F5F80936302CFBFCF91089529
:101060008230E8F4E82FF0E0EE0FFF1FEC59FD4F5F
:1010700071836083813041F0809169008C7F842B83
:1010800080936900E89A089580916900440F551F84
:10109000440F551F837F842B80936900E99A08953C
:1010A0001F920F920FB60F9211242F933F934F93DD
:1010B0005F936F937F938F939F93AF93BF93EF93C0
:1010C000FF938091640290916502892B29F0E09151
:1010D0006402F09165020995FF91EF91BF91AF9184
:1010E0009F918F917F916F915F914F913F912F9140
:1010F0000F900FBE0F901F9018951F920F920FB672
:101100000F9211242F933F934F935F936F937F938D
:101110008F939F93AF93BF93EF93FF93809166025A
:1011200090916702892B29F0E0916602F0916702A5
:101130000995FF91EF91BF91AF919F918F917F9111
:101140006F915F914F913F912F910F900FBE0F9034
:101150001F9018951F920F920FB60F9211242F9384
:101160003F938F939F93AF93BF9380916902909128
:101170006A02A0916B02B0916C023091680226E085
:10118000230F2D3720F40296A11DB11D05C029E8BB
:10119000230F0396A11DB11D20936802809369025D
:1011A00090936A02A0936B02B0936C0280916D02DF
:1011B00090916E02A0916F02B09170020196A11DF4
:1011C000B11D80936D0290936E02A0936F02B09355
:1011D0007002BF91AF919F918F913F912F910F908E
:1011E0000FBE0F901F9018952FB7F8946091690269
:1011F00070916A0280916B0290916C022FBF0895EA
:101200003FB7F89480916D0290916E02A0916F02A9
:10121000B091700226B5A89B05C02F3F19F001962A
:10122000A11DB11D3FBF6627782F892F9A2F620F0E
:10123000711D811D911D43E0660F771F881F991F47
:101240004A95D1F70895CF92DF92EF92FF92CF9314
:10125000DF936B017C010E940009EB01C114D104F2
:10126000E104F10489F00E946E0D0E9400096C1BDC
:101270007D0B683E734090F381E0C81AD108E10805
:10128000F108C851DC4FEACFDF91CF91FF90EF908A
:10129000DF90CF900895789484B5826084BD84B542
:1012A000816084BD85B5826085BD85B5816085BD61
:1012B000EEE6F0E0808181608083E1E8F0E010827A
:1012C000808182608083808181608083E0E8F0E0BB
:1012D000808181608083E1EBF0E0808184608083A5
:1012E000E0EBF0E0808181608083EAE7F0E08081DC
:1012F0008460808380818260808380818E7F808310
:101300008081806880831092C1000895833081F0CD
:1013100028F4813099F08230A1F008958730A9F047
:101320008830B9F08430D1F4809180008F7D03C083
:10133000809180008F7780938000089584B58F77A7
:1013400002C084B58F7D84BD08958091B0008F77F1
:1013500003C08091B0008F7D8093B0000895CF933B
:10136000DF9390E0FC01E458FF4F2491FC01E0572B
:10137000FF4F8491882349F190E0880F991FFC0169
:10138000E854FF4FA591B49182559F4FFC01C59140
:10139000D4919FB7611108C0F8948C912095822355
:1013A0008C93888182230AC0623051F4F8948C9126
:1013B000322F309583238C938881822B888304C0BD
:1013C000F8948C91822B8C939FBFDF91CF910895DD
:1013D0000F931F93CF93DF931F92CDB7DEB7282FC4
:1013E00030E0F901E859FF4F8491F901E458FF4FCB
:1013F0001491F901E057FF4F04910023C9F08823AD
:1014000021F069830E9486096981E02FF0E0EE0FE8
:10141000FF1FE255FF4FA591B4919FB7F8948C91AF
:10142000611103C01095812301C0812B8C939FBF54
:101430000F90DF91CF911F910F910895CF93DF937C
:10144000282F30E0F901E859FF4F8491F901E45861
:10145000FF4FD491F901E057FF4FC491CC2391F095
:1014600081110E948609EC2FF0E0EE0FFF1FEC5572
:10147000FF4FA591B4912C912D2381E090E021F4B0
:1014800080E002C080E090E0DF91CF910895FC0100
:10149000818D228D90E0805C9F4F821B91098F731C
:1014A00099270895FC01918D828D981731F0828DD6
:1014B000E80FF11D858D90E008958FEF9FEF08955F
:1014C000FC01918D828D981761F0828DDF01A80F4C
:1014D000B11D5D968C91928D9F5F9F73928F90E06E
:1014E00008958FEF9FEF08958EED9BE0892B49F0D3
:1014F00080E090E0892B29F00E94DE0B81110C9492
:1015000000000895FC01848DDF01A80FB11DA35ACE
:10151000BF4F2C91848D90E001968F739927848F13
:10152000A689B7892C93A089B1898C9180648C930A
:10153000938D848D981306C00288F389E02D8081F5
:101540008F7D80830895CF93DF93EC01888D88236E
:10155000C9F0EA89FB89808185FD05C0A889B98920
:101560008C9186FD0FC00FB607FCF5CF808185FFFB
:10157000F2CFA889B9898C9185FFEDCFCE010E9469
:10158000820AE7CFDF91CF910895CF92DF92FF9249
:101590000F931F93CF93DF931F92CDB7DEB76C01EC
:1015A00081E0D60158968C9358975B969C915B97F7
:1015B0005C968C915C97981307C05096ED91FC91C6
:1015C0005197808185FD2EC0F601038D10E00F5FDD
:1015D0001F4F0F731127F02EF601848DF81211C0E2
:1015E0000FB607FCF9CFD6015096ED91FC915197BB
:1015F000808185FFF1CFC60169830E94820A6981DB
:10160000EBCF838DE80FF11DE35AFF4F6083D601C6
:101610005B960C935B975296ED91FC91539780816A
:1016200080620CC0D6015696ED91FC91579760836D
:101630005096ED91FC91519780818064808381E088
:1016400090E00F90DF91CF911F910F91FF90DF906D
:10165000CF900895BF92CF92DF92EF92FF92CF93F7
:10166000DF93EC016A017B01B22E60E874E88EE141
:1016700090E0A70196010E946F0D215031094109A8
:1016800051095695479537952795E889F98982E05C
:101690008083211580E1380798F0E889F989108264
:1016A00060E472E48FE090E0A70196010E946F0D64
:1016B000215031094109510956954795379527958C
:1016C000EC85FD853083EE85FF852083188EEC89BF
:1016D000FD89B082EA89FB89808180618083EA8903
:1016E000FB89808188608083EA89FB8980818068AA
:1016F0008083EA89FB8980818F7D8083DF91CF9110
:10170000FF90EF90DF90CF90BF9008951F920F92BF
:101710000FB60F9211242F938F939F93EF93FF9304
:10172000E0918102F09182028081E0918702F09144
:10173000880282FD12C0908180918A028F5F8F7330
:1017400020918B02821751F0E0918A02F0E0EF586D
:10175000FD4F958F80938A0201C08081FF91EF91A8
:101760009F918F912F910F900FBE0F901F90189502
:101770001F920F920FB60F9211242F933F934F9306
:101780005F936F937F938F939F93AF93BF93EF93E9
:10179000FF9381E792E00E94820AFF91EF91BF914F
:1017A000AF919F918F917F916F915F914F913F91F9
:1017B0002F910F900FBE0F901F90189581E792E028
:1017C0000E94470A21E0892B09F420E0822F089526
:1017D000109274021092730288EE93E0A0E0B0E0E1
:1017E0008093750290937602A0937702B09378026B
:1017F00089EA91E0909372028093710285EC90E007
:1018000090937E0280937D0284EC90E0909380021E
:1018100080937F0280EC90E090938202809381021B
:1018200081EC90E0909384028093830282EC90E0BC
:10183000909386028093850286EC90E090938802D4
:101840008093870210928A0210928B0210928C026F
:1018500010928D02089508950E944B090E942B0C4E
:101860000E94AA00C4E7DAE00E94E2002097E1F3B8
:101870000E94740AF9CFCF92DF92EF92FF920F93FA
:101880001F93CF93DF936C017A01EB01E60EF71EF5
:1018900000E010E0CE15DF0561F06991D601ED9111
:1018A000FC910190F081E02DC6010995080F191FE8
:1018B000F1CFC801DF91CF911F910F91FF90EF9071
:1018C000DF90CF9008956115710581F0DB010D90D7
:1018D0000020E9F7AD0141505109461B570BDC01CF
:1018E000ED91FC910280F381E02D099480E090E07D
:1018F00008950C94630CDC01ED91FC910190F08152
:10190000E02D099465EB71E00C94630C0F931F9329
:10191000CF93DF93EC010E94630C8C01CE010E94F7
:10192000820C800F911FDF91CF911F910F9108952D
:101930008F929F92AF92BF92CF92DF92EF92FF92DF
:101940000F931F93CF93DF93CDB7DEB7A1970FB659
:10195000F894DEBF0FBECDBF7C01C42EE52FCB01B6
:10196000D22E19A221E02D1510F02AE0D22E8E01E0
:101970000F5D1F4F8D2C912CA12CB12C6C2D7E2F27
:10198000A50194010E946F0D8C2DD29E8019112407
:10199000015011098A3014F4805D01C0895CF8019E
:1019A0008083211531054105510521F0C22EE32F19
:1019B000CA01E4CFB801C7010E94630CA1960FB61B
:1019C000F894DEBF0FBECDBFDF91CF911F910F9175
:1019D000FF90EF90DF90CF90BF90AF909F908F904F
:1019E0000895CF92DF92EF92FF920F931F93CF93C0
:1019F000DF93EC016A017B012115310579F4E8815F
:101A0000F9810190F081E02D642FDF91CF911F913A
:101A10000F91FF90EF90DF90CF9009942A3031051D
:101A2000E9F477FF1AC06DE20E947B0C8C01442719
:101A30005527BA014C195D096E097F092AE0CE01CC
:101A40000E94980C800F911FDF91CF911F910F91F1
:101A5000FF90EF90DF90CF9008952AE0B701A601A4
:101A6000CE01DF91CF911F910F91FF90EF90DF900A
:101A7000CF900C94980C9A01AB01662757FD6095A6
:101A8000762F0C94F10C0F931F93CF93DF93EC01FF
:101A90009A01AB01662757FD6095762F0E94F10CE5
:101AA0008C01CE010E94820C800F911FDF91CF919B
:101AB0001F910F9108952115310541F4DC01ED913D
:101AC000FC910190F081E02D642F09940C94980C06
:101AD0009A01AB0160E070E00C945B0D0895A1E207
:101AE0001A2EAA1BBB1BFD010DC0AA1FBB1FEE1F98
:101AF000FF1FA217B307E407F50720F0A21BB30BE3
:101B0000E40BF50B661F771F881F991F1A9469F75E
:101B100060957095809590959B01AC01BD01CF01BA
:101B20000895EE0FFF1F0590F491E02D0994F894AD
:101B3000FFCF00000E0380004E6F6465200020720E
:101B40006561647900544F505345435245545041A8
:101B500053535752440073656E64696E6720746F07
:101B6000206E6F646520002C206D6573736167655E
:101B7000205B005D0041434B2072656365697665BB
:101B80006421006E6F2041434B2072656365697666
:101B900065640072656365697665642066726F6D61
:101BA000206E6F646520005D2C2052535349200045
:101BB00041434B2073656E7400000000000B073A30
:101BC00002E2065A07C0075D03B00177032904EE5D
:101BD00002E007D301B50100000000C50A3B0C4735
:101BE0000A600A520AA30A0D0A006E616E00696E4D
:101BF00066006F7666002E00FFFFFFFFFFFFFFFF0E
:101C0000FFFFFFFFFFFFFFFFFFFFFFFFFFFFFFFFE4
:101C1000FFFFFFFFFFFFFFFFFFFFFFFFFFFFFFFFD4
:101C2000FFFFFFFFFFFFFFFFFFFFFFFFFFFFFFFFC4
:101C3000FFFFFFFFFFFFFFFFFFFFFFFFFFFFFFFFB4
:00000001FF
